:1000000012C0189518951895189518951895189563
:100010001895189518951895189518951895189578
:100020001895189518958FE58DBFC0E4E6E24E2E21
:1000300084E08EBFD4E0F4E05F2EEEEFF3E0A0E6C4
:10004000B0E084B7082E877F84BF8FE181BD80E058
:1000500081BD88278D933197E9F789E189B980E0DF
:1000600080BD88E18AB9662489E189B980E080BDD4
:1000700086E880BD01D380E081B988E480B984E05E
:1000800086BF8F9A41D1C5D0CDD081E080939B00AF
:1000900000919B00033010F009F00FC0979A84E69E
:1000A00090E0FCD1979884E690E0F8D1ABE9B0E01D
:1000B0008C918F5F8C9308F4EBCF979AC9D1ABE901
:1000C000B0E08C9300919B00013009F089C0C4D14D
:1000D000ACE9B0E08C9300919C00013609F00AC0B5
:1000E000E8E5FCE0C5D1CAD17CD0ECE8FCE0C0D1A9
:1000F000C5D176C0023609F00AC0EEE8FCE0B8D1FE
:10010000BDD199D0ECE8FCE0B3D1B8D169C00336D9
:1001100009F02EC0E2ECFCE0ABD1B0D105D1E9E9A9
:10012000F0E0D190E0808FEFE7FE8827F82E082FCF
:100130000AD3ADE9B0E038D3E4E5FCE07BD3EDE9E8
:10014000F0E0E2D243D3EDE0F0E0ADE9B0E06CD511
:10015000E6EEFCE08DD1AEE0B4E0EDE9F0E0D4D223
:10016000ACD17ED18BD1ECE8FCE082D187D138C014
:10017000073609F006C0EEEFFCE07AD17FD11DD141
:100180002FC0013009F021C06ED081E080939B0028
:1001900000919B00013110F009F016C0AEE0B4E010
:1001A000EBE9F0E0A190BB24E2E6F0E0AA0CBB1C76
:1001B000EA0DFB1DC5D454D161D1ABE9B0E08C91FF
:1001C0008F5F8C9308F4E4CF0BC0023009F008C0B5
:1001D000ABD0AEE0B4E0E9E9F0E0BAD441D14ED121
:1001E0006DCF5FD210EE65D210E063D25AD211EE1D
:1001F00060D27AD2ABE9B0E01C9355D2E2E3FDE0E5
:1002000037D1AEE0B4E0EBE9F0E0A9D429D136D1A2
:10021000089547D210EE4DD212E04BD216E449D2E7
:1002200042D208953ED210EE44D211E042D211E003
:1002300040D239D2089535D210EE3BD211E039D2F6
:1002400030D211EE36D250D2ABE9B0E01C932BD2B3
:10025000E8E4FDE00DD1AEE0B4E0EBE9F0E07FD4FE
:10026000FFD00CD108951DD210EE23D210E021D280
:1002700011E51FD218D284E690E010D112D210EE10
:1002800018D212E016D20DD211EE13D281E0809373
:100290009B0000919B00003110F009F021C026D294
:1002A000A1E6B0E01C9322D2A0E6B0E01C93A1E648
:1002B000B0E09C91A0E6B0E08C91ABE9B0E0AD90ED
:1002C000BB24A2E6B0E0AA0CBB1CAA0DBB1D8D93FB
:1002D0009C93ABE9B0E08C918F5F8C9308F4D9CFFD
:1002E00005D2A1E6B0E01C93FFD1A0E6B0E01C93DC
:1002F000DAD1A1E6B0E09C91A0E6B0E08C91A4E850
:10030000B0E08D939C93089580E0E3E3D6D3A6E814
:10031000B0E00C9380E0E3E35BD3A7E8B0E0E5EA6C
:10032000F0E098E082D4089580E080938F0080E030
:10033000E3E3A7D26CEC80E0E3E3BB27A6E121E096
:100340002A93CBD264E480E0E3E3BB27A6E121E07B
:100350002A93C3D28EEE92E0A1D080E0E3E3A7E837
:10036000B0E0BED36EEB80E0E3E3BB27A6E121E083
:100370002A93B3D280E0A0E9B0E0E3E329E02A9336
:10038000D2D288E0E0E9F0E055D4402F0091980007
:10039000041709F00BC0A1E9B0E09C91A0E9B0E01E
:1003A0008C91A9E9B0E08D939C9306C08EEC9FEFF1
:1003B000A9E9B0E08D939C930895E6E5FDE058D05F
:1003C000AEE0B4E0E6E8F0E0CAD34AD057D087E028
:1003D000E7E8F0E02FD4ABE9B0E00C9340919B004C
:1003E00000918E00041709F02CC0EEE6FDE040D02D
:1003F00045D0E0E9FDE03CD088E080939C0040914E
:100400009C0001E0041710F009F016C0AEE0B4E063
:10041000ECE9F0E0A190BB24E6E8F0E0EA0DFB1D7A
:10042000E8D31ED0ECE9FDE023D080919C00815000
:1004300080939C0008F0E3CFECE8FCE019D01ED0DC
:1004400004C0EEE9FDE014D019D00895F894FFCF70
:1004500081E05F9B882708955F9BFECF8CB1089554
:10046000AEE0B4E08D91882311F00BD0FBCF08955E
:10047000DDD1802D11F005D0FBCF08958DE001D0A6
:100480008AE05D9BFECF8CB908953197F1F708950E
:10049000689462F80895E89462F80895EF93FF93E2
:1004A000EE27E82BE92B31F0E0EAFFE03197F1F796
:1004B0000197D1F7FF91EF9108958DE207FD8D939C
:1004C0008F2D881F802F881F8F57082F6894F7F86B
:1004D000802F87FF15C080958395082F80E38D932B
:1004E0008EE28D93802F815228F080E38D9399279F
:1004F0009C93089544270A95802F09F192D01FC03C
:10050000805230F09EE49D9381E48D939D93EFCFD4
:100510004427DF92EF92FF920F938FE1801B11F03F
:10052000082F7FD085D09EE29D930F91FF90EF9092
:10053000DF9044270395003209F4D7CF27D03F93AB
:10054000E2ECF5E038E12F2D1E2D0D2DFF24EE24D9
:10055000DD244427000F111F221F88F42F923F92A1
:1005600065D1102C63D1202C61D1302C5FD1319713
:10057000410DD21CE31CF01C3F902F9001C033961C
:1005800031963A9539F73F9107D0B3CFDD0CEE1C89
:10059000FF1C0A95D9F70895002719E058D08F93CA
:1005A000802B11F0039501C08F911A95B9F7802F18
:1005B000882309F49ACF8F91805D8D930A95D9F79E
:1005C00096CF0065CD1D80B2E60E40597307A0ACF2
:1005D000B90350D6DC01286BEE0094357700CA9A37
:1005E0003B0065CD1D00B2E60E0059730700ACB9A3
:1005F0000300D6DC01006BEE0000357700009A3B6B
:100600000000CD1D0000E60E000073070000B903D6
:100610000000DC010000EE000000770000003B005D
:100620000000F694E794D79447950A95D1F708957A
:1006300000270DD08F9303958F2D8E298D29842B24
:10064000C1F78F91805D8D930A95D9F750CF1F9395
:100650000F93002710E2440FDD1CEE1CFF1C001F4F
:10066000802F9AE0890B10F0082F43951A9599F77F
:10067000802F0F911F910895AC9AAD9AA498A598D8
:100680000895689446BF8F939F9388279927019672
:1006900021F046B747FFFBCFE8949F918F9162F816
:1006A000089544EAEECF44E946BF46B747FDFDCF83
:1006B000089513B944E8E5DF8F939F93882799271E
:1006C000019669F041B1487F483FD1F3E894483141
:1006D00039F0483229F0403419F0403509F0689477
:1006E0009F918F9162F8089544E801C044ECC9DFFE
:1006F00013B141B1487F483FE1F326F06894487058
:1007000009F0E89462F80895D190E190F190019198
:100710000895102F90E8FF0C001F0927990FF794F8
:100720001078652F90E8440F551F5927990F47956A
:10073000607800380895FF0C90E89027110F979586
:10074000F794092F0895102FBD2CDE2CEF2CF02EDE
:1007500011234AF4B094D094E094F0949FEFB91A26
:10076000D90AE90AF90A0EE1FF2039F4FE2CED2C32
:10077000DB2CBB240850C2F723C032F00A95BB0C17
:10078000DD1CEE1CFF1CF9CF01D0D5CFB7FE0895BC
:1007900090E8B91611F4D0FE08959FEFD91AE90A2E
:1007A000F90A09F403950895DD92ED92FD920C93F8
:1007B00008959FE7092FF92A9FEFD92EE92E089572
:1007C000DD24EE24FF24002711270895A2DFC1F3C2
:1007D0005038B1F31627005850580894051F12F4EA
:1007E00018F4E7CF08F0ECCF0AD0FF202AF0BB0CBA
:1007F000DD1CEE1CFF1C9FCF0F5FDBF29CCF9F9296
:100800009924AA24BB24992788E1990CAA1CBB1C13
:10081000DD1CEE1CFF1C30F4920EA31EB41ED91E6C
:10082000E91EF91E8A9589F79F900895C89531961B
:1008300000200895FBDF202DF9DF302DF7DF402D5C
:10084000F5DF502D089591E0882321F08894991FB9
:100850008A95E9F7892F90950895883018F01196B8
:100860008850FBCF08950181082B01831281192341
:100870001283EF93FF93E4E0F0E007DEFF91EF9146
:10088000089506DEFF27DFDFEEDFEF93FF93ECE74F
:10089000F7E0FBDDFF91EF91182B12830923018311
:1008A000EF93FF93E4E6F1E0F0DDFF91EF9110812B
:1008B000182359F4EF93FF93ECE7F7E0E6DDFF919F
:1008C000EF911081182309F0E6DDEF93FF93ECE739
:1008D000F7E0DBDDFF91EF910895B5DFFF27299168
:1008E0005D9148E0C0DFEF93FF93E4E0F0E0CDDD01
:1008F000FF91EF91579510F4182B1283EF93FF930C
:10090000ECEEF0E0C2DDFF91EF91182B1283EF9334
:10091000FF93E4E0F0E0B9DDFF91EF914A9511F724
:100920002A95F1F608958FDFFF27299148E0552792
:100930009ADF09230183EF93FF93E4E1F0E0A5DD63
:10094000FF91EF9188941081182309F0089457952E
:10095000EF93FF93E0EBF0E098DDFF91EF914A9584
:1009600039F75D932A9511F708957DDF09230183F7
:10097000EF93FF93E4E1F0E088DDFF91EF91E894DD
:100980001081182309F06894EF93FF93E4ECF0E0F2
:100990007CDDFF91EF91089566DFEF93FF93E4E034
:1009A000F0E073DDFF91EF9116F4182B1283EF93B3
:1009B000FF93ECEEF0E069DDFF91EF91182B1283CD
:1009C000EF93FF93E4E0F0E060DDFF91EF91089595
:1009D00033273093A4003093A10053DF0EF458C0A6
:1009E0003091A10030FD54C066276093A300639549
:1009F0006093A20021E050EF48E074DFB6DF31F9E8
:100A0000B4DF32F9632F6670663009F441C060309C
:100A100019F031FB40D025C06091A2007091A40074
:100A20006717B1F0C0F48F939F93862F8A95A5EA3C
:100A3000B0E013DF08DF7C9178236894772329F4F2
:100A4000E8946091A2006093A3009F918F9109C0E8
:100A5000689421D006C0E8941ED06091A2006093F3
:100A6000A3009ADF6091A20063956093A2006134B5
:100A700009F0C4CF6091A3006093A4006623E894BA
:100A800009F4689430F93093A100E89462F808956D
:100A9000689462F808958F939F93A5EAB0E08091DF
:100AA000A2008A95DADECFDE7C9116F4782B01C0A5
:100AB00079237C939F918F9108958F9389DF8F91F4
:100AC000A0E0B0E056F011968F93AF93BF9385DF0F
:100AD000BF91AF918F910EF0F6CF0A2F1B2F089583
:100AE000AF93BF93EF93FF9338E0E5EAF0E00D9109
:100AF00001933A95E1F7FF91EF9130E43093A40030
:100B000033273093A10069DF38E0BF91AF91E5EA68
:100B1000F0E00D914191041719F43A95D1F7089539
:100B2000B7DC0895000F111F221F331F0895009591
:100B30001095209530950F5F1F4F2F4F3F4F089511
:100B4000019110810EC001911191219130810BC052
:100B50000191108117FF05C03FEF2FEF04C0008106
:100B600011272227332737FF03C0E1DF8DE28D9362
:100B7000CF93DF93CF92DF92EF92AA24BB24CC24B1
:100B8000DD24EE2440E2CAE0DD2755E093E38881CE
:100B9000890F87FD9F7083FD907F891B89935A95EC
:100BA000A9F7C0DFAA1CBB1CCC1CDD1CEE1C4A959F
:100BB00051F7E894EFE0FF2782910ED0EB30E0F799
:100BC0001EF068948A2D0CD088278D93EF90DF90CB
:100BD000CF90DF91CF910895982F829501D0892FE2
:100BE0008F70805D26F0803309F4089568948D93AA
:100BF000089541E003C042E001C044E0E40F8827CB
:100C0000F81F8291982F829505D0892F03D04A959D
:100C1000C1F707C08F708A3008F0895F805D8D93BF
:100C2000089588278D93089594E081918D939A95E6
:100C3000E1F7089500276CE8719198E006957795A3
:100C400077FF18F477FD08F006279A95B9F78A958B
:100C500099F708950000003F46756E6B74696F6EDA
:100C60003A2053524620556C747261736368616C0C
:100C70006C6D6F64756C2053572D5265766973697E
:100C80006F6E206175736C6573656E00000046754C
:100C90006E6B74696F6E3A2053524620556C7472B5
:100CA00061736368616C6C6D6F64756C204C696313
:100CB000687473656E736F72206175736C657365AC
:100CC0006E0046756E6B74696F6E3A20445331380E
:100CD000533230205465706572617475726D65733E
:100CE00073756E67000047656D657373656E65208B
:100CF00054656D70657261747572203A2000467596
:100D00006E6B74696F6E3A2031576972652D4B6F47
:100D10006E66696775726174696F6E206175736C58
:100D20006573656E20756E642061757367656265B5
:100D30006E00536F667477617265205265766973D1
:100D4000696F6E203A2000004C69636874776572A1
:100D500074203A200000416E7A61686C2031576936
:100D600072652D446576696365733A2000004352CD
:100D7000432064657320656D7066616E67656E659E
:100D80006E20524F4D2D436F646573204F4B000012
:100D9000524F4D2D436F6465203A2000200043528E
:100DA000432064657320656D7066616E67656E656E
:100DB0006E20524F4D2D436F6465732046414C5356
:040DC00043480000A4
:00000001FF
